:020000041004E6
:20000000008A000841060410414204104542041000000000000000000000000000000000C1
:20002000000000000000000000000000614204100000000000000000634204106542041095
:2000400067420410694204106B420410154404106D4204106F4204107142041073420410DE
:200060007542041077420410794204107B4204107D4204107F4204108142041083420410F0
:20008000000000000000000000000000000000000000000000000000000000000000000060
:2000A000000000000000000000000000000000000000000000000000000000000000000040
:2000C000000000000000000000000000000000000000000000000000000000000000000020
:2000E000000000000000000000000000000000000000000000000000000000000000000000
:2006400072B600200021002200230024002500260027104880F308880F4810490860BFF331
:200660004F8F03F036FE0E4FB8470E4A0E4C00231360121DA242FBD30C4B0D4A0D4C15686C
:200680002560121D241D5B1E002BF8DC00F0ECFEFEE700BF008A00080000041008ED00E0F4
:2006A00085420410004A0008C15E00080400000000FD0410004A0008004A0008FF8900089D
:2006C00000000000000000000000000000000000000000000000000000000000000000001A
:2006E0000000000000000000000000000000000000000000000000000000000000000000FA
:200700000000000000000000000000000000000000000000000000000000000000000000D9
:200720000000000000000000000000000000000000000000000000000000000000000000B9
:200B00004630335F48513030315F535746425F303030382E303030312E303000000000006E
:200B20004170722020372032303232000000000030393A34333A3436000000000000000087
:200B4000303030303030303030303030000000000000000000000000000000000000000055
:200B6000000000000000000000000000000000000000000000000000000000000000000075
:200B8000000000000000000000000000000000000000000000000000000000000000000055
:200BA000000000000000000000000000000000000000000000000000000000000000000035
:200BC000000000000000000000000000000000000000000000000000000000000000000015
:200BE0000000000000000000000000000000000000000000000000000000000000000000F5
:200C00001111111111111111FFFFFFFFFFFFFFFFFFFFFFFFFFFFFFFF1111111111111111D4
:200C20002222222222222222FFFFFFFFFFFFFFFFFFFFFFFFFFFFFFFF2222222222222222A4
:200C40003333333333333333FFFFFFFFFFFFFFFFFFFFFFFFFFFFFFFF333333333333333374
:200C6000000000000000000000000000000000000000000000000000000000000000000074
:200C8000000000000000000000000000000000000000000000000000000000000000000054
:200CA000000000000000000000000000000000000000000000000000000000000000000034
:200CC000000000000000000000000000000000000000000000000000000000000000000014
:200CE0000000000000000000000000000000000000000000000000000000000000000000F4
:200D000000002110422063308440A550C660E770088129914AA16BB18CC1ADD1CEE1EFF1D3
:200D20003112100273325222B5529442F772D662399318837BB35AA3BDD39CC3FFF3DEE393
:200D40006224433420040114E664C774A44485546AA54BB528850995EEE5CFF5ACC58DD553
:200D60005336722611163006D776F6669556B4465BB77AA719973887DFF7FEE79DD7BCC713
:200D8000C448E5588668A7784008611802282338CCC9EDD98EE9AFF9488969990AA92BB9D3
:200DA000F55AD44AB77A966A711A500A333A122AFDDBDCCBBFFB9EEB799B588B3BBB1AAB93
:200DC000A66C877CE44CC55C222C033C600C411CAEED8FFDECCDCDDD2AAD0BBD688D499D53
:200DE000977EB66ED55EF44E133E322E511E700E9FFFBEEFDDDFFCCF1BBF3AAF599F788F13
:200E00008891A981CAB1EBA10CD12DC14EF16FE18010A100C230E3200450254046706760D2
:200E2000B9839893FBA3DAB33DC31CD37FE35EF3B1029012F322D232354214527762567292
:200E4000EAB5CBA5A89589856EF54FE52CD50DC5E234C324A0148104667447642454054452
:200E6000DBA7FAB79987B8975FE77EF71DC73CD7D326F2369106B016576676761546345612
:200E80004CD96DC90EF92FE9C899E9898AB9ABA94458654806782768C018E1088238A328D2
:200EA0007DCB5CDB3FEB1EFBF98BD89BBBAB9ABB754A545A376A167AF10AD01AB32A923A92
:200EC0002EFD0FED6CDD4DCDAABD8BADE89DC98D267C076C645C454CA23C832CE01CC10C52
:200EE0001FEF3EFF5DCF7CDF9BAFBABFD98FF89F176E367E554E745E932EB23ED10EF01E12
:200F000000050000B918041001050000191604100205000019190410030500005D190410BF
:200F200004050000851A041005040000551A041006050000E9180410E51F0410190088137D
:200F400001020301ED1F041019008813010203026D2004101900881301020303F91E041025
:200F6000000000000000000010010203000000004D1E0410000000000000000011010203C5
:200F800000000000652804100D2A04102D2A041022010203000000004D2F04100000000042
:200FA000000000002702000000000000592A0410CD2B0410E32B0410310102000C00000003
:200FC000A134041000000000000000003402000000000000253104109F3204104733041015
:200FE0003602000001000000913304101534041071340410370200000300000089200410D1
:2010000000000000000000003E01020300000000BD35041000000000000000002E02000056
:2010200000000000854004100000000000000000280300000000000001000000ED1E04108C
:201040000000000000D101000000000021D00100000C04107EF12000200C04107FF120004D
:20106000400C041080F12000F52B04103F2C041000FF0C000100007101FF00487200000095
:20108000452E0410932E041004030400010000710103044A10000000C12C0410E52C0410EF
:2010A00001FF0C000100007101FF014A100000000000051098F10700040000002000051079
:2010C00099F107000400000000000000000000000000000040420F0040420F0040420F00C8
:2010E00040420F00060700009F070000DF0700008F070000DF0700009F070000DF070000BE
:201100001A070000000000008F070000DF0700000A070000000000000400000049160410AA
:201120008316041019210410C5220410AB21041083220410352304104523041055230410AC
:201140004D230410D9240410FD26041049190410511904108D1904109B190410091A041016
:20116000E73C0410AD3704103F3D0410493D0410DD190410553E0410613E0410CD3E041093
:20118000B51A0410C31A0410CB1A0410D31A0410E91A0410F11A0410AF1B0410D71B041067
:2011A000FF1B04103F1C041000000040000400000103060507090000010706020308050A05
:2011C0000102030A0F000000010A0B0C070D0E000A07030006010703080500000107030669
:2011E0000508000000010203040506000000000014410410C05E0008010000000600000037
:201200000001020304050607080C101418203040080C1014182030400001020304050607D6
:2012200008090909090A0A0A0A0B0B0B0B0C0C0C0C0D0D0D0D0D0D0D0D0E0E0E0E0E0E0E34
:201240000E0E0E0E0E0E0E0E0E0F0F0F0F0F0F0F0F0F0F0F0F0F0F0F0F0000008412041076
:201260004C5E0008D8120410E01204106C5E00080000000000000000F012041001020201CA
:2012800001000100F412041000000000F412041001007808080000000000000100005340FB
:2012A00000800000010000000000524002077808081304100007080000000000020000074B
:2012C0007808000000000000000001078008000001000000000000000000000000010100FB
:2012E00000000000000000000100000000FF0000000000001000F4010207020002070201D2
:20130000FF00D00704000000E0070000DF0700000000000000000000000000000000000026
:2013200000000000000000000000000000000000000431400100000000000000080000002F
:20134000150000000000000000000000000000000000000000000000000000000000000078
:201360000000000000000000000000000004314000000000010000000E00000015000000D4
:2013800000000000000000000000000000000000000000000000000000000000000000004D
:2013A0000000000000000000040000000000000000000000000000000000000010B581B033
:2013C0002349244C244A0B68A34200D1234A01689002C30F01D1080E05E0012B02D108028A
:2013E000000E00E0084693085840D0231840D3021B0E5A24634018188B0F0C0E63400C0B76
:2014000063408C086340DB07DB0F490019430138F2D1D0070DD50802000E0B0E1B04184321
:201420000B061B0C1843FF231B0219400904084300E00846504000F007F80090684601B08D
:2014400010BD07480021704700BA0021704700BF040800080101FEFEDCB6F23AD7B7C13AEE
:201460007856341272B6704700B500F002F8002000BD00B502F0F4FF00F010F80121062023
:2014800000F032F80121084600F02EF80121002000F02AF800F008F800BD00000149002041
:2014A00008707047B25A000870B581B000F0F2F800F091FF00F078FA534908780028F5D0CE
:2014C000524908780728F1D282008118504A49008A185049C0000818537A4468107AC11A08
:2014E000C9B29818A047E1E770B507284CD28300C218474B52009B181C7A082C0ED20022E0
:2015000003E09D5C8D4202D00132A242F9D3D2B2A24203D19954197A013119723A4C3B49E8
:201520002278002A07D12278072A2DD2227888540120207028E0374DC200AA18567800221E
:2015400017E08B5C834217D0DB00EB185B78B3420DD2237803E04D1EED5CCD54013B934218
:20156000F9D8DBB2C85423780133237004E00132D2B223789A42E4D323789A4204D12278E0
:20158000885420780130207070BD10B5072839D28300C2181E4B52009B185A7A13E09C5C60
:2015A0008C420ED100219954597A8A420ED1013159721A7AC9B2914208D1002159721972C3
:2015C00004E00132D2B21C7AA242E8D31A7A002A18D10D4913E00D4B9C5CA0420DD104E057
:2015E000D018407898540132D2B2087801388242F6D308780138087004E00132D2B20B7813
:201600009A42E8D310BD00BFB25A0008B45A0008BC5A0008000F0410F0B505460E460024D4
:201620000DE02F5D39460120FFF7AFFF7A1ED2B2022A03D203489200105880470134B44299
:20164000EFD3F0BD1C11041000B59649002008709549087095490870954902015218013086
:2016600010731328F8D3C0B200014018FF210173002002F03BFF0021C943002002F06AFF8E
:2016800000BD00B588490020087002F081FF02F0A0FF00BDF0B586B0834F0022029238789C
:2016A00000286FD0834C104602F088FF064620680021864200D2012105917A492660002570
:2016C000097801913978049159E0019A784910014418217B0091D1B2E07A0391012808D10F
:2016E0000598012843D10020E072606886423ED305E06068864202D20598012837D1A17ACB
:20170000607AFFF7F1FE207A012809D1206880196060B04201D9002000E00120E07226E047
:20172000387860490138387008780199884204D1217B5C480091017014E00499481E8542B6
:201740000298034606D15A4A00018018FF210173009107E0564A00018118207B08730090A6
:20176000DAB203925149019A087820730A700398C0B202900098C0B201900135EDB20498DB
:201780008542A2D306B0F0BDF9B581B00F4602931146019004467D20C00004F0D1FC810010
:2017A000401A49014018C60004D139462046FFF79BFE41E000240136204602F0FFFE394ACA
:2017C00000902546117811E0394C09010C19617A0198884207D1A17A8F4204D101983946F1
:2017E000FFF7D3FE06E0217B0135EDB22E4803789D42E9D3142D1FD22B4801788D420FD172
:201800000131017029482A4A01780C01A418227B0270244802782273017001986072A7727F
:20182000029820720098266031186160814201D9002100E00121E17201B0F9BDF0B581B004
:20184000184A00240094167826E0194F3201D5196A7A90421CD1AA7A914219D1FFF795FE44
:201860001149087801380870002C03D10D49287B087008E0C0B2FF21844200D0297B009820
:201880000001C01901730949087828730E7007E000962E7B0134E4B2034B1A789442D4D3C1
:2018A00001B0F0BD065B0008055B0008045B0008085B0008B85D0008F0B505460E460024A2
:2018C0000DE02F5D39460020FFF75FFE7A1ED2B2042A03D203489200105880470134B44247
:2018E000EFD3F0BD24110410F0B505460E4600240DE02F5D39460620FFF747FE7A1ED2B253
:20190000052A03D203489200105880470134B442EFD3F0BD34110410F0B505460E4600245C
:201920000DE02F5D39460220FFF72FFE7A1ED2B2032A03D203489200105880470134B44215
:20194000EFD3F0BD4811041000B500F0E4FE00BD00B5002000F0E8FE00BD0000F0B505460F
:201960000E4600240DE02F5D39460320FFF70DFE7A1ED2B2082A03D20348920010588047A4
:201980000134B442EFD3F0BD5411041000B500F015F809490120087000BD00B500F01AF823
:2019A00005490020087000BD00B503490878012801D100F0F0FE00BD485C000810B51349A0
:2019C0000C7802F03FFA012C03D107210420FFF78BFD10BD00B502F039FA00BD00B502F082
:2019E00098F800BD60B581B0094E3578012D08D10093084D13460A460146287801F088FE5A
:201A000000E0002001B060BD704700BF4A5C0008495C00084B5C000800B50B4A10700B4A99
:201A2000117006210420FFF75FFD00BD06490870704707490870704700B5104600F0B4F926
:201A400000BD014908787047495C00084B5C00084A5C0008F0B505460E4600240DE02F5D5D
:201A600039460520FFF791FD7A1ED2B2032A03D203489200105880470134B442EFD3F0BD7A
:201A800074110410F0B505460E4600240DE02F5D39460420FFF779FD7A1ED2B20A2A03D298
:201AA00003489200105880470134B442EFD3F0BD8011041000B57F490320087000F0C6FE0F
:201AC00000BD00B500F0C3FE00BD00B500F0A2F900BD00B578490878012802D100F064FEE5
:201AE00001E000F07DFE00BD00B501F0EAFA00BDF0B585B06A46002003AF019078803B1F57
:201B0000191F981DFFF76EFF04907A88694649C90546002A11D0694C694F21780801C019E0
:201B200082811F46E0C0049AC270012201318270C9B2052004F022FB21700020604A010178
:201B40008C18A17B01292CD15E490878012805D05D490878012801D100F048F8564DA1687C
:201B60005A480A782B783E2A0DD1E27B002B01D1427000E0027023686268A08900F084FA0E
:201B80000020A07311E0002B0FD1E27B42705048626802604F4823680360A08900F0A0F80D
:201BA000EEE70130C0B20528C8D305B0F0BD00B582B0474B474A01A9881EFFF713FF454894
:201BC000026843480168022000F017FA3D490220087002B000BD00B53F4A0123032104204B
:201BE000FFF7D2FD38490120087000BD00B503210420FFF723FE344A0020107000BD00B5A5
:201C00002D490878002819D02A4A1078810040183249800040184068804701280ED10421F9
:201C20000846FFF70BFE244A0020082110700320FFF75AFC06210420FFF756FC00BD70B53C
:201C400004210846FFF7FAFD1A49244C08788100401880000019806880471E490B681C4971
:201C6000144E0A68014630788500401980000019007B00F073F8104E0020307070BD30B524
:201C800014480C4D0368124878210268287884000019124C80000019007B00F05FF830BDE4
:201CA000044A1078810040180C4980004018007B704700BF9E5C00089C5C0008BC5D000834
:201CC0004C5C00089D5C0008A15C00089F5C0008144A0008104A0008404B4C005C0F04102D
:201CE000F1B581B001900D4616461F460024A200A1184F4A89008A182878117B88421FD13F
:201D0000002101B48B184B485B7B0078834201BC08D001310329F4D33B4632467F2100F061
:201D20001DF811E044493B460C701068324600900198294601B40198844601BCE04703E0AC
:201D40000134E4B20B2CD2D30B2C05D13B4632462878112100F002F801B0F1BD30B5374D52
:201D60000C462978364D002901D1697800E02978002909D1112C07D3122C14D9312C12D00C
:201D80007E2C01D37F2C0ED994707F2150701170032018800821FFF7A7FB782C03D0062134
:201DA0000420FFF7A1FB30BD00B5224A117801291ED0224A1178002901D0002818D1214954
:201DC0000878002808D1204A012303210420FFF7DBFC1C4901200870174A1078810040181F
:201DE000134980004018007B312801D101F071F8114A1078810040180D4980004018007B4A
:201E0000112802D100F06AF803E0102801D100F021F900BD00B500F022FA00BD054908706C
:201E2000704706490870704702490878704700BF5C0F04109D5C00089E5C00089C5C0008AA
:201E40009F5C0008A15C0008404B4C00F0B516461F460D464978264B4C06640E00221A7048
:201E6000511CC9B2012906D303D003290FD314D001E0022813D30132052AF1D31D4A50687C
:201E800080476878000614D5FFF7C4FF16E0194B1978A142EFD0122102E00228EBD0132138
:201EA0003B4632461120FFF759FF11490120087004E03A463146204600F001F8F0BD00B52B
:201EC000512348700B700220108008210320FFF70BFB06210420FFF707FB00BD00B504495F
:201EE0000878002801D1FFF795FF00BD704700BFA25C000838100410F2B581B015464A7854
:201F00005106490E00915A491E4600220A70594C531CDBB2012B1BD305D0032B06D336D042
:201F2000042B38D014E0022833D311E000239900CF1A5149BF007F18FF7A00998F4201D10B
:201F4000237002E00133032BF1D3DBB2032B35D00132052ADCD32078474F8200101A8000BB
:201F6000C059804720788200101A8000C0194349C07A087001994A7812062CD5012827D011
:201F80003F4A012303210420FFF7FEFB28E00228DED0132113E0002723789900CB1A364997
:201FA0009B005B18F918354B097A1B788B4202D00137032FF0D3F9B20329C9D11221334683
:201FC0002A461020FFF7CAFE29490120087007E0FFF720FF04E032460098294600F00DF844
:201FE00001B0F2BD00B501F093F800BD00B525490020087001F07CF800BD70B515460C46E4
:2020000000218B005A1A1C4B9200D218D37A83421CD15021217060709088010AA170E07068
:20202000D68831460520400204F08AF82071304604F07EF860710620288008210320FFF79C
:2020400053FA06210420FFF74FFA02E001310329D7D370BD00B506490878002805D10749C0
:202060000878012801D1FFF7D5FE00BD704700BFA35C0008A45C0008380F04109D5C00087E
:20208000404B4C009C5C000870B54E7875066D0E0024611CC9B2012906D303D003291AD37D
:2020A0001DD001E002281CD30134032CF1D330061CD515490878012825D0144908780028E9
:2020C00021D1134A012303210420FFF75DFB11490120087017E0002DE6D0122102E00228EB
:2020E000E2D013213E20FFF739FE0CE07E20107055700220188008210320FFF7F5F906218F
:202100000420FFF7F1F970BD9D5C00089C5C0008404B4C00A15C000830B5394900200870B2
:202120000120FFF77BFE374C00202070022000F063FA05461020FFF779FC3348854204D170
:2021400001202070FFF772FC15E0304A30491068884205D1052020700120FFF767FC0AE051
:202160002C49884205D1092020700120FFF75EFC01E0002020702078002810D0FFF759FCA4
:2021800002F043F800F050F8022000F015FAFFF758FC012808D10220FFF740FE04E0012012
:2021A000FFF73CFE00F001F830BD00B5FFF73CFE01281DD1032000F01FFA1349114A884270
:2021C00001D0002000E001201070002810D002F01CF800F029F810490120104A08700023FF
:2021E00004211846FFF7D0FA0D490120087003E002F00BF800F018F80A490120087000BD2C
:20220000AC5C0008A55C0008AA55AA55848B00080110CCCC0111CCCCA65C0008204E0000C5
:20222000004A0008A75C000800B5FFF71BF901210420FFF759F901210320FFF755F9012149
:202240000220FFF751F900BD00B503F080FD002001F092FE244801210843804700BD00B587
:2022600002210320FFF740F902210120FFF73CF902210846FFF738F902210020FFF734F97C
:2022800000BD00B519490878012816D1184A002002211070FFF728F902210320FFF724F945
:2022A00002210120FFF720F902210846FFF71CF902210020FFF718F903E0022801D1FFF730
:2022C000CEFF00BD00B509490878012804D100200870FFF7B9FF05E006490878012801D0FB
:2022E00002F0F0F800BD000000080110004A0008A65C0008014A000800B50C49086000F01D
:2023000001F800BD00B50949086802280DD108490878012809D104210020FFF78FFA044AA2
:2023200000201070032000F047F900BDA85C0008A65C000800B5062002F097F968490120A8
:20234000087000BD00B500F009F800BD00B500F01AF800BD00B500F00CF800BD00B5614AAB
:2023600003201070604A1168604A106802F0C0F900BD00B55C4B1A685C4B19685C4B1868E0
:2023800002F013FA00BD70B558490D6856490C6857490E68FFF784FC56490870E00FC007DA
:2023A00002D00120640064085349087053490878002806D152490D60524908604F49012067
:2023C0000870484B022018704D4B22463146186800F027F870BD00B541490878012805D157
:2023E00002F05EFA022801D102F093F900BD70B5444B044600201860404B0D461646187004
:20240000FFF74EFC3B4B404A40491870611A914205D232462946204602F026FA00E00020D7
:2024200070BDF1B581B03A4B0D46184614461A780026002A01D1202C29D231461F1D202A10
:2024400008D2A14214D26B5CBB5401320270D2B20131F4E72F4B621A49191A6020243D4634
:202460002D4A1160274A067011680919116028E021490978012901D1114612E0194A167060
:20248000264A1178264A1078FFF72EF814E0214AE106C90E1160641A6119E1E7FF237B54F0
:2024A00001312029FAD3174B012620241968891819603D460021017016480021012E016048
:2024C00008D10F4A01981168091911602246294602F0FAF801B0F1BD00B500F0BDF800BDF4
:2024E000B75C0008B65C0008184A0008B05C0008B85C0008BD5C0008B45C0008B55C0008BB
:202500001C4A0008244A00080100030000000110C45D0008204A0008C05C0008BC5C0008E3
:20252000C55C000801490868704700BF244A00080120704710B5084C2070084C2170084C12
:202540002270084C2360084C2360084C02982060074C0398206010BDC55C0008BC5C000849
:20256000BE5C0008B05C0008808B0008B85C0008184A000800B583B00021019102912F49E6
:202580000022D24313460CC12D4B00210328197005D102AB6A4601A9012000F037F8284A02
:2025A00000991078002805D0264B01981860029A02F08AF803B000BD00B583B0204A002386
:2025C000019302931370022802D11F490B6011E003280FD102AB6A4601A9022000F016F85C
:2025E00017490878002805D0164A01981060029902F07EF803B000BD022804D0032804D124
:202600001249086801E010490868704730B5012808D0022811D10A4A012010700B480A4604
:202620000B4908E0064D062028700448094C0460064C0C6008211060196030BD284A000811
:20264000B65C0008808B0008840900080080051020000000AA55AA5530B51D4C00252078FA
:20266000022811D11B480268002A06D01A4B19681A4B1868FFF7D5FE1BE0194908780128E7
:2026800004D11848057001E0032809D1164A25701570164A1178164A1078FEF725FF08E05E
:2026A000124A1178124A1078FEF71EFF0E4A2570157030BD00B50F4A002010600A4A10706E
:2026C0000D4A11780A4A1078FEF70EFF00BD00BFB65C0008204A0008C05C00081C4A0008A2
:2026E000B45C0008B55C0008C45C0008BC5C0008C55C0008808B0008BE5C000800B50E4AF6
:20270000012303210220FFF73FF8002001F008FC03F01DFB00BD00B503210220FFF78EF8CE
:20272000002001F029FC00BD00B5C82001F04DFC03F00DFB00BD00BFA086010000B503F089
:202740002BF903F004FB094802F045FB0021084602F04EFA00BD00B50221002000F0D2FFC1
:202760000121002002F044FA00BD00BF5C12041000B584B0417901AA1170811D0291016880
:202780000079009110726946022002F050FA04B000BD0020704700B502F01AFA02F021FA90
:2027A00002F00EFA00BD000000B5FFF768FA2849012008700220FFF734FB264A002304214C
:2027C0000846FEF7E1FF2449087881004018234980004018007B312801D100F07BFB00BD03
:2027E00000B51D4A1078810040181C4980004018174A007C117881420CD2FFF740FA14488C
:20280000144A017801310170002304210846FEF7BBFF03E00A210420FEF766FE00BD104859
:20282000704730B5002305E0D41A0419CD5C013C257001339342F7D330BD10B5002302E064
:20284000C45CCC540133013AFAD210BD70477047C65C0008404B4C009E5C00085C0F041040
:20286000FF0F0000FFB582B002907148002100910170704C0099645C012C04D0032C16D0CB
:20288000072C53D002E00298032815D300980130C0B200900628ECD3674E0498306067480B
:2028A0000124059901606648002505609FE00298441EE007C70F01D0132142E0614861084B
:2028C0000124017001975F4805786D00AC4235DA0398015D0E020134E4B2005D064300259D
:2028E000594BEA009B189A88964216D1DB79012B0AD100F0EAFB002806D133210191514808
:2029000004786400E4B2DEE7504B4948DD550378013701330370FFB202E00135052DDFD317
:2029200001980028EBD10134E4B2CCE740480178444800788142A9D0312102E00199002964
:20294000A4D0059B049A2220FFF708FA5CE03F4F3D4B7A5DD2009A189079019011689288B1
:20296000002913D03168120A0A5531687A5D0134D2009A1892880A55316801347F5D611872
:20298000FF000246F858FFF758FF24E0D12109028A420FD13268D121115531687F5D01340A
:2029A000FF00DF19BF880F550134FFF73DFA3768385510E026498A4213D13268D0211155E7
:2029C00031687F5D0134FF00DF19BF880F553168013401270F551A4B019824181F683F1839
:2029E0001F6009210420FEF77FFD0135EDB2154800788542ABD30120FFF713FA154A002304
:202A000004210846FEF7C0FE02B0FFBD0A4B622118680A4B01701968094B1A68094B1878C9
:202A200040001018013008800120704710207047CC5C0008B0110410304A0008344A0008A9
:202A4000C85C0008CD5C000840100410D05C000821D00000A8610000FDB582B00290C24807
:202A60000C46002101700091C04EC14FC149009A895C062900D381E0012900D283E003D0A5
:202A800003292AD33CD07EE0029804287BD213216BE0FFF7C9F9012801D1312165E0A178AE
:202AA00000220D02E1780D4311468800431ADB009B191B899D4201D1397002E00131032933
:202AC000F3D3C9B2032900D1312211464BE000F0FCFA002857D1332147E000213B789A00C4
:202AE000D31ADB009B19CA186378127B934202D001310329F2D3C9B2032944D1122134E043
:202B00003B789A00D31ADB009B195B890298984201D0132127E0002125E0397800228B0004
:202B2000591AC900891901920989FF200002814218D39148814215D89048211D0422FFF708
:202B400070FE21468E4808310422FFF76AFE8C4B19688A4B8B4A186800F0D5FD002801D1CF
:202B600031210191019900290DD0049B039A3120FFF7F4F87C480121017025E00729A6D35D
:202B800087D00829C9D000980130C0B20090082800D26BE77C49029A0A807C490C607C4914
:202BA000039A0A607B490498086039788800411AC900895988470120FFF733F9764A002312
:202BC00004210846FEF7E0FD02B0FDBD00B5684A10788100081A6549C0004018406880477D
:202BE00000BD634A10788100081A6049C0004018007D704700B582B060490868FFF798FCC1
:202C0000002817D1654B012018700320FFF7F4FC092101300AD00023019300930A22042073
:202C2000FFF788FC0320FFF7C7FC06E00420FEF75BFC02E05A490120087002B000BD30B576
:202C400082B0564D00242878012836D324D0032814D332D14E4B1968454B18788200101ABA
:202C6000424AC00080180F300522FFF7E6FD494B1868052101802C7001241EE0019400948E
:202C800023460A2209210420FFF754FC0320FFF793FC0120287010E039490A22086801900B
:202CA00036480094092103680420FFF743FC02210620FEF719FC03202870204602B030BD01
:202CC00000B501210520FEF70FFC364A01201070354A00201060354A092110700420FEF786
:202CE00003FC00BD30B582B02E4900240878012800D2A4E02BD003287DD300D191E0042883
:202D000000D09CE0224B2A4C1868411D601C0122FFF793FD1E4B1868811D20460122FFF77B
:202D20008CFD1B4B1968124B18788200101A0F4AC00080180F300522FFF77FFD154B072179
:202D40001868184B018000201870012477E0FFF766FD16490A781449084D0B682968534365
:202D6000074DC918023825E0345D000868100410365D0008B811041001FF0000384A0008B8
:202D80003C4A0008C75C0008945A0008404A0008444A0008484A0008A8610000385D00081C
:202DA000355D0008395D00084C4A0008375D00087C4A00082B68834204D90120C0021B1A86
:202DC000013202E0184623462246534D2860534D2B60534D534B2A70019000910A2209210C
:202DE0000420FFF7A7FB03210620FEF77DFB4E4D0220287023E048494A4B0A2208680090B6
:202E00000921042001F06FF802210520FEF76CFB424A01201168002900D103204249087022
:202E20000DE000943F4B0A220921042001F05BF803210520FEF758FB3B49042008702046B2
:202E400002B030BD00B582B0384A1068013017D0374B012018700320FFF7CEFB0921013072
:202E600003D00420FEF740FB11E00023019300930A220420FFF75EFB0320FFF77BFB06E0DC
:202E80002B4A0220092110700420FEF72DFB02B000BD00B5274B1968274B18788200101AEB
:202EA000264AC00080180F300522FFF7C6FC244B062118681E4B01801878012803D0022876
:202EC00005D1012000E002201A4A11684871012000BD704710B5184A10788100081A17491C
:202EE000C00040180089FF210902884212D115480478012C0ED10320FFF77EFB013000D0E1
:202F00000224114A002014700E4A092110700420FEF7EAFA10BD00BF4C4A00083C4A0008D5
:202F2000375D00087C4A0008395D0008000801103A5D0008444A0008365D00086810041014
:202F4000484A0008355D0008385D0008F0B51E460D46497814464A06520E00235C49C95C8C
:202F600001292AD307D0032913D318D00A2937D00F293DD021E002281FD2132133462246A9
:202F80002720FEF7EBFE5349002008705249087096E0012A11D0022A0FD01221EEE700210F
:202FA000012A02D1022805D105E04C4F3F780237B84200D013210029E0D10133052BCDD3C7
:202FC0000127012A36D144490878002816D1FEF738FA434A03C20843F9D03E48077011E000
:202FE000022AEAD13B4F39780029E6D12421C5E73C4F39780129E0D13721BFE73848002128
:203000000A4606C06878012856D1344B6770672020701D7832482A46A11CFFF70EFCA81CFD
:20302000308008210320FEF75FFA06210420FEF75BFA45E02A480021FEF7C0F90021274BB8
:203040001A78914222D24B19425C9B789A421AD025493525087801300870C0B202280BD9CB
:20306000224A3625002305210420FEF78DFB1D481D4907700020087033462246294627202E
:20308000FEF76CFE1CE00131C9B2D8E712490F70104900200870687802280DD1672020709F
:2030A00002206070308008210320FEF71DFA06210420FEF719FA03E008210420FEF714FA90
:2030C000F0BD0849002008707047034908787047C01104103E5D00083C5D000818110410BA
:2030E000504A00083D5D00083B5D00088096980000B508490878012802D10220FFF7FCF8B0
:20310000054900200872054908700549087000BD704700BFA65C0008485D00083C5D0008B0
:203120003B5D0008F4B582B01E460D460021884B5B5C012B57D00A2B04D362D00C2B73D3A4
:2031400000D185E001310729F1D3821E814C82482146028092B2A81CFFF76FFB7F490C6057
:203160007F49029808607F4806607F480378687898427FD17D4A012010707D4A14607D4CA0
:20318000FFF7D0F97C4A216840181060724A11887A4A7B4B11601868401818606368984214
:2031A00003D10120C007084310600120FEF739FE744A002304210846FEF7E6FA6F490868FA
:2031C0006B4901900A22086800906B48092103680420FFF7AFF904210620FEF785F96A4903
:2031E0000220087059E0634A00249368DB0705D4022800D21324002CA4D034E00328F9D397
:20320000F9E75C4C0023277AFF070AD5564A17786A78013FBA4205D0594A17686268974296
:2032200000D124231C46E6E74F4A002314786A78013CA2420AD0524A4E4C17683F1862684C
:20324000023F974202D97123002222721C46D2E7454A6C7813789C4200D173E7013B9C42F3
:2032600000D16FE773243346029A21463620FEF775FD12E04449032008703B49581E0870CB
:203280000120FEF7CEFD3F4A002304210846FEF77BFA09210420FEF727F902B0F4BD30B519
:2032A00082B0394D00242878012849D338D0032811D345D12B4A02211068294A01801068A4
:2032C000762101701068284A1178417001312C701170012434E02849086825490860FFF78D
:2032E00021F92A4A1168401A24490860FFF71AF926490860194803681F4820490360086849
:203300001B4901900A220868009009210420FFF711F903210620FEF7E7F8012028700FE078
:2033200016490A2208680090134809210368042000F0D9FD02210520FEF7D6F80320287062
:20334000204602B030BD0B490020087272207047C81104107C4A0008965A0008704A0008BC
:20336000744A00086C4A00083F5D0008405D0008644A0008485D0008684A0008604A0008B1
:20338000584A0008A8610000425D00085C4A0008F0B581B000243949095D032910D00A2904
:2033A00015D1374E00213578002D05D0354F3D68354F7E68B54200D02421002903D106E050
:2033C000012804D013213720FEF7C8FC20E00134032CE0D32D4802602D4829490360002054
:2033E00008702C4901200870FEF71BFD2A4A002304210846FEF7C8F900200090274B0A222C
:203400000921042000F06FFD03210520FEF76CF801B0F0BD30B582B01E4D00242878012893
:2034200015D0022821D11948016877220A70184A116803220A80194902684B78537000686A
:2034400009788170104804722C7001240DE00194009423460A2209210420FFF76BF80521F3
:203460000620FEF741F802202870204602B030BD0549002008721020704700BFD0110410B6
:20348000405D0008584A0008485D00087C5A0008805A0008445D0008A8610000465D000813
:2034A000F9B500900C46174600253E49495D06293DD201290AD0032913D0052929D03BE03A
:2034C000FFF703FE002837D133212AE0009805280AD331E06178002919D1A178442916D15B
:2034E0002AE000980B2827D013211AE02E4EE11C30460422FFF795F9E11D301D0422FFF7D2
:2035000090F92A4A03CE00F0FEF8002814D1312107E0254800218268D20700D5222100291F
:203520000AD0019B20783A46FEF718FC39E00729C6D3CFD00829D9D00135062DB5D3FFF7B2
:203540006EF9194A91680322914301221143164A9160174A01211170164A00211160164A91
:203560000446116001210520FDF7BEFF74213970202179700021CA190220451AED00083D79
:2035800026462E41967001310229F4D3019A0421118008210320FDF7A7FF06210420FDF7B0
:2035A000A3FFF9BDD4110410485D0008C75C00083F5D0008584A00085C4A0008F9B50090A8
:2035C0004B4817460C46FF2101706078A27801020A430026474DB300991B890049198988B9
:2035E0008A4202D14248067002E00136022EF1D300264149895D062906D201290AD0032952
:2036000022D0052932D00DE0072929D306D0082932D007E00098042820D303E034480178F0
:20362000FF2934D00136062EE3D3314801788A00511A89004D59A178982935D101214903D9
:20364000284601F055F82BE0294801788A00511A89004919C98800988842E3D0132117E058
:20366000FFF733FD0028DDD1332111E0234801780129D7D122210BE01D4801788A00511A52
:2036800089006A584919097A515C5529CAD13121019B3A462E20FEF761FB28E001F039F8FD
:2036A00001F0FEF80228F9D0154EE01C31460422FFF7C3F820223146284601F005F801E08D
:2036C00001F027F801F0ECF80228F9D0019A032111806E21397061787970A178B97008215D
:2036E0000320FDF701FF06210420FDF7FDFEF9BD545D0008B0100410DC110410405D000890
:203700007C4A0008704700B5FEF771FE00BD0000F4B581B0B94A1578B94A0E46B94C107800
:20372000A84225D01F46691CC9B2032002F008FDB24A631C117061784C1EE407E40F1C7082
:203740002B03E818B04B019AC3181360AF4C6B00079A1B5B33808B01C818AD4B4000C018AB
:203760001060AC48490040183860AB48405D1BE0AA48017801290FD100210170019AA8488F
:203780001060A84A10883080079AA7481060A748A74A1860107807E00020308007999C4864
:2037A00008609C481860012001B0F4BDF0B583B0002000F049FC041C00D16EE19D4A036803
:2037C00011789D4A09018E1831688B4202D071688B42EDD1307B022805D3A079717B8842B1
:2037E000E6D1012000E00020944F38706579082DDED301198A79F02111403029D8D801B465
:2038000070688F4EC01A00D0012033780290012B01BC00D9DCE00B1C49D10291082DC7D8C5
:2038200011070D0F0095C3D00722111A8D42BFDC734E01990029357809D10019C0793E28AB
:2038400005D1764A01210291117075480AE07D490878002802D0184600F0BBFA2903681806
:20386000694940183A78A11D51184A1C0021535C4354009B01319942F9D302981A46002802
:203880000BD16249680042526348019A4255681CC1B2032002F054FC03E06248644E019993
:2038A0000280317000210120FEF7B6F880E7019A002A00D17CE7102937D1002000F089FACC
:2038C000387801198A791207CB79120D06311A430823181A824200D26AE75B48824204D983
:2038E0003221002000F0DBF862E7584B0020187057480260424A107802038018424A821826
:2039000054488B1C0021026003E0585C50540131C9B238780624201A8142F6DB4E4A302168
:203920001060002000F0BBF842E7202900D03FE7444A1178022900D03AE7444A1178013170
:203940000907090F0019117082791207120F91423AD1414A3F4CC31D116820680D18002056
:2039600006E0195C29541168013111600130C0B2374C2668B14210D239780724611A8842A9
:20398000EFDB364842683648002301780320FDF7FBFE3449042008700AE7002000F019FADE
:2039A000174E1A4A23683178480083521A48012242540131C9B2032002F0C2FB3170002191
:2039C0000120FEF729F8F3E6002000F002FAEFE6302900D0ECE60198002800D1E8E6032B6D
:2039E00000D0E5E61007000F40D11F49088004203070002000F00FF9DAE600BFE85D00085D
:203A0000595D0008E85D00080C0B0008A45A0008080A00089C5A00085A5D00086E5D0008CC
:203A2000040A0008985A0008000A0008A05A0008585D00086D5E0008F8100410615D0008F0
:203A4000605D00085D5D0008FF0F00005E5D0008845A0008645D0008685D0008D41004109A
:203A6000E41004105F5D0008AC5A0008022810D0BC4AF521FF31108888420AD20130108017
:203A8000B9484268B948002341780320FDF77CFE8EE6002000F0A9F98AE603B0F0BD10B552
:203AA00084B001AA1070B24B0C46082151701A7841005118AF4A0901511889680091694695
:203AC00000F0A1F9AC4A6846811D107842180C5400235370F42393700330C0B202E000222F
:203AE0000A5401300828FAD3302C0DD1A34901200870A34802689D48002301780320FDF78E
:203B000043FEA049032008706846FEF731FE04B010BDF0B584B000263446304635469A4A3F
:203B20009A4F11784B00FB181F88002F06D01D808E018B19964E3C465B009E190139C907B7
:203B4000C90F11700130C0B2002C07D10228E6D390480488002C5CD005808F4E01AA157034
:203B6000834A8449107800014018806800906946284600F048F9804B07221978501A84424F
:203B800018DC01AA0820507088188470C21C294602E0705C50540131E0B28142F9D3197887
:203BA0000723591AC9B201E0155401308842FBD301201EE068460630220A10231A43425485
:203BC00008184470821C01AB08205870284603E0335C13540130C0B206277B1A9842F7DB7F
:203BE0006E490E606E490B806E490D706E4902200C806E4908706846FEF7BAFD6C49012066
:203C000008705948026859482B4641780320FDF7BBFD04B0F0BDF0B586B0644D01242878D5
:203C200004285ED103AA00201070514A51491078000140188068029002A9002000F0E3F8B6
:203C40005849087801300007000F08704A49544F524E0B7802A95918202210438871CA1D9A
:203C6000398830680E180196002007E0019E0131365C398089B216540130C0B20726F61A86
:203C8000B04205DA01B448480088814201BCEDD303AF08237B70F6B202E000231354013039
:203CA000B042FAD3404A1088814202D300240520287002A8FEF75CFD0020FEF76AFD00280E
:203CC00001D0002C0BD13A4901200870264802682648002341780320FDF756FD01E0012C55
:203CE000AED006B0F0BD00B524480178012901D1022101702D490878012805D0022810D0BB
:203D000004280AD0052819D1002000F06EF8012200211046FDF790FE10E00020FFF77BFF74
:203D20000CE0032008702249022008700E4842680E48002341780320FDF726FD00BD00B519
:203D4000002000F006F800BD00B5002000F032F800BD00B50B4A1178002901D000F039F83E
:203D600000BD00BFAC5A0008DC100410E41004106D5E0008F8100410615D00085D5D00083A
:203D8000D41004105F5D0008EA5D00089C5A0008080A0008A05A0008000A0008885A000802
:203DA000B05A00086D5D0008AE5A0008605D00086C5D000810B51B4904460878002807D087
:203DC000204600F012F8214600220120FDF734FE10BD00B5144A00201070144A1070144AF7
:203DE00003201178FDF72AFD00BD00B5114A00201080114A10700B4A10700D4A032051788C
:203E0000FDF71CFD00BD0D4A40011018027B022A03D3407B8871012000E0002008490870FB
:203E2000704700BF6C5D00085D5D00085F5D0008E4100410AC5A0008605D0008F8100410BE
:203E4000615D000800B5FEF779FC00BD00B5FEF782FC00BD2A49012008702A49087070472D
:203E6000F0B5284D2878012804D002281ED00120287026E024480468402C03D9403C0460B4
:203E8000402401E002202870204E1D48204F328803783868214600F0F1F8194F30801C494F
:203EA0000020387008680019086007E0194A002028701178184A1078FDF716FB2878002807
:203EC00003D002210520FDF70FFBF0BD00B5104A10680E4A11880F4A018011780E4A107861
:203EE000FDF702FB00BD10B50B4C2070094C21700A4C2270064C2360034C0298206010BD8F
:203F0000745D0008705D0008905A0008725D00088C5A0008755D0008715D0008765D0008B1
:203F2000002828D172B60E4A01201060022010600C4A0121C9071068084310600A4A0B489B
:203F40001060084A1021106808431060084A0121C907106808431060014A0320106009E0FD
:203F600040C0264010C0264008C026405019000000C0264062B67047002824D172B60D4B7C
:203F800001201860022018600B4B0020186058600A4B0B4918605868400840005860586867
:203FA000102290435860586808405860014B0320186007E040C0264004C026400CC02640F4
:203FC000FFFEFFFF62B60020704700280DD072B6044901200860022008600120486003207E
:203FE000086001E040C0264062B67047F0B581B01E4F1F4C3A7813011B190C689D1D042643
:2040000001B42088288002340235013E01BCF7D1047900681C711860087958710132D2B27F
:20402000032A00D332463A7005210320FDF75CFA01B0F0BD00B50F4A107801301070042101
:204040000320FDF751FA00BD0B4A084B11781878814209D0064B0801C0180131C9B20329D9
:2040600000D30021117000E0002070477C5D0008805D0008B05D00086E5E000800B500F0C0
:204080002FF800BDF0B54C788026264067067F0E00256C1CE4B2012C02D0022C04D00AE09F
:2040A000032808D2132102E0052F04D912212820FDF754FE13E00135022DEAD3802E0ED072
:2040C000682010704878507088789070032018800821FDF709FA06210420FDF705FAF0BD92
:2040E00010B50A4C012B00D0144622460AE00478130A63401402A2B2DBB2054C5B001B5BA8
:204100005A4001300139F2D2104610BDFFFF0000000D041000000000F0B583B00023029304
:2041200000286DD0002A6BD001238B4014680193002C01D1436000E083603C4C137A041B1E
:204140003B4DE40924016519DE06F60E1F27042908D2CBB2DB002C689F40BC439E40264301
:204160002E6008E00B1FDBB2DB006C689F40BC439E4026436E60019CE643846C536934408A
:20418000DB07DB0F8B4023438364C46C93693440DB07DB0F8B402343C364D36900934B005D
:2041A0001C4610340327C56CA740BD43009FBF07BF0FA7402F43C764546800948C000F274E
:2041C000456CA740BD43009F3F073F0FA7402F434764D7680325046C9D40AC43BD07AD0FED
:2041E0009D40254305644369019B43614369836912693340D207D20F8A401A43826101E0FA
:204200000C490291029803B0F0BD10B500242101081B094980004018024601790068083200
:20422000FFF77AFF0134022CF1D310BD000031400000304001005A003013041000007047D1
:20424000FEE7FEE704207146084202D0EFF3098001E0EFF3088000B5004FB847434204104B
:20426000FEE7FEE7FEE7FEE7FEE7FEE7FEE7FEE7FEE7FEE7FEE7FEE7FEE7FEE7FEE7FEE7EE
:20428000FEE7FEE710B564488208D2B2002004E0624C830001301C595C5061499042F7D308
:2042A000604A1160402210684422086410685E4A48641068000A00024021084310605B4927
:2042C0001068084010605A4A012010600220106010BD00B5574B002018605860564B0121B0
:2042E0001860564B0904186888431860544B186888431860534B1868884318601868012170
:20430000090588431860186801218904884318604D4B002018604D48302100F02FF84B481A
:20432000322100F02BF84A4B186801231843484B01211860414B4904186808431860404BAF
:204340001868084318603F4B0121090418680843186018680121090508431860374B012107
:204360000904186808431860354B18680843186008200222052100F01BF800BD4A09012A7A
:2043800009D30ED0022A12D1403901228A40816D114381650BE001228A40016D11430165C6
:2043A00005E0203901228A40416D11434165704730B5284B8000C31818680725A8434C07D6
:2043C000640F2043186018680124E407204318608807C00E9207130EFF2585408340002938
:2043E00002DB8A08104C04E00A07120F083A9208194C920012191468AC431C431460002977
:2044000007DBCA06D20E154B0949012090401860086030BD704700BF800000000000041090
:20442000008A000808ED00E000E400E0FF00FFFF00E100E0500021405800214000132040B6
:2044400080132040000024400C00214000002140C8002140008020401CED00E080E200E003
:2044600030B5034A034801241060A407024D05E0C05D0008A81104100004004072B60320CA
:2044800080020019ED30FF300F210160084A0020A050084A13200002A05000200122120373
:2044A000A05005482860286804482860286807E0180C00003C1000000F00FF830000FF83D9
:2044C00062B630BD05490020C043086048600449002008600349044808607047001826404C
:2044E000081026400CED00E00400FA0510B572B60F4AF02110680F4A08400021C943116054
:204500000D4A0123FF33002418C20C4A090D11600B4A022111600B4A772111600A4A012156
:2045200014600A4AC9071460014A084310600FE080033940A0033940C4033940CC033940DA
:20454000B0033940D4033940F80339408803394062B610BD10B50C4672B6084A0121C907FF
:20456000106808431060064A1460064A00201060054A102110680843106007E080033940CE
:20458000A003394088033940C003394062B610BD72B6074A1168074A1068000A00021060A3
:2045A0000846034A0121C9070843106004E000BF80033940C803394062B6704710B572B614
:2045C00001490C6802E000BF8803394062B6204610BD72B6164A17491068400040080840FD
:2045E0001060154A0020C0431060144A00201060134A1449106808400121FF3108431060E4
:204600005068000A000250600F4AC32189001068084310600D4A1068000A000210600C4A8C
:20462000322010600B4A106840084000106013E080033940FFFFF8BFA0033940880339402F
:20464000C4033940FF00FFFFCC033940B0033940D4033940F803394062B67047062801D90E
:204660001F2001E00849085C704710B5074A117B884224D1064A074C117800290CD10122F8
:20468000032304210BE000BFE4110410F0110410EC5D0008185E0008FE22FC23FB2162700B
:2046A000A370E17072B6204600F052FA62B6E088FFF7D4FF0021002803D17B4901E0FF20A2
:2046C00000217A4A118010BD30B5794D02242C70784D01242C70784C784BE260A06003C315
:2046E0002161204600F04EFAE088FFF7B7FF30BD10B56F4B0222704C1A706E4B03221A7048
:20470000A060E160204600F0FDF9E088FFF7A6FF10BD00B500F007F869490878012801D16B
:2047200000F02BF800BD00B5664B624A986900281BD11968002907D01078012804D15A69B8
:20474000186900F064F817E01078032806D1D869196A814202D900F06DF80DE054490020AA
:2047600010700870FDF778FF06E000201070504901200870FDF79EFF00BD00B5504A5248E7
:204780001178012910D1002111704268002A05D04E4B0068196800F014F805E045490A70CF
:2047A00043490A70FDF758FF00BD30B5404D02242C70404D454B2C70044612C300F001F8F6
:2047C00030BDF0B5144600230125ED02AA4204D92C469E00375877500133A608B342F8D3E4
:2047E000AA4206D29B0002E0C55CCD5401339342FAD33648111BB30081604168C9184160F7
:204800000168091901602E4801210170F0BD30B52C4C0D4600F01DF9616920232031616120
:204820002169203121610021202D00D3E91A2160A06130BD10B5044600F059F801210907E6
:20484000611A1F221204914208D2214A0121C9036118914205D20121C90301E00121490320
:204860000A191C4905C110BDF0B506460C4600250F18FDF715FA002C10D0042C0ED9164909
:204880008E4206D315498F4203D8032109048C4203D9342802D1E00600D101252846F0BD63
:2048A00003490878704700BFA5A50000145E0008785D0008775D0008185E0008005E000855
:2048C000165E0008F05D0008F85D0008F45D000800001F10085E000800000110000004108F
:2048E0006F490868012108436D490860704700B500F009F8011C04D06A4A0121904200D13E
:204900000421084600BD70B50026674C3546674A214603466CC10120FF30FFF756FB01F0D8
:2049200016FA63482246012100F009F804460120FF30FFF74AFB01F00AFA204670BD10B51F
:2049400081B0036804465B48002B11D55A4BE2601A686B46009219800099A160E16900296B
:2049600003D45149086800F00BF852498842F5D0524A116801221143504A116001B010BD24
:20498000010F0A2901D1002062E04D4A2921490490421ED24B4A90420FD24B4A904257D0DA
:2049A0004A4A904252D04A4A904233D0494A904201D1481C4CE048484AE0484A90422FD022
:2049C000474A9042F7D829D03E4A904224D9C81C3EE0444A90420BD2434A904227D823D0C5
:2049E000424A90421ED0364A9042E4D1881D2FE03F4A904227D03F4A904221D03E4A9042B8
:204A00001BD03E4A904215D0364A9042D3D108460A301DE008461BE0881C19E0081D17E0EF
:204A2000481D15E0C81D13E00846083010E0084609300DE008460B300AE008460C3007E076
:204A400008460D3004E008460E3001E005200005704700B5114600F011F81F4988420BD087
:204A6000011C09D00F49884201D1042104E01E4A0121904200D10321084600BD10B50A4ACE
:204A800000231F4C5360052393801460906000230748D160D3710121FFF751FF10BD00BF5B
:204AA00000F4244002005200305E0008000100140000224002005000EC110410080024406E
:204AC000910000F0040000F00F005200090000A0010000F0030000F0FFFF00000A0000F07B
:204AE000060000F0A60000F0A40000F0920000F0BB0000F0B20000F0AA0000F0A80000F095
:204B00000001010610B50E4A04460E491068884201D0052011E0A068C20401D002200CE0F9
:204B2000E168002908D0084A09181160074A1060FFF780FE002800D10020E08010BD00BF0D
:204B4000405E00083C3CA55A105E00080C5E000810B504464078012805D1A078032802D174
:204B6000E078042801D0062005E0FFF7B9FE0349034808600020E08010BD00BF405E000877
:204B80003C3CA55A10B50C4A04460C491068884201D005200DE0A068420701D0022008E093
:204BA000E168002904D02269FFF731FE002800D10020E08010BD00BF405E00083C3CA55ADD
:204BC00000B58D4A10684168006800F06DF900BD00B5894B186808224168006800F07FF901
:204BE00000BD00B584490868006800F089F900BD70B5814A1068002460C8012904D30BD0DF
:204C000002290ED0012410E0287900F046FA3146284600F082F908E03146284600F087F918
:204C200003E03146284600F06FF9204670BDF0B58DB005460E46002400F001FB002804D133
:204C40000621052000F017F90124002E05D10621012000F010F90124BAE0002C00D0B7E04C
:204C600031790991B1680691317B37680491002F05D4624862493840884205D809E0614951
:204C8000B8008008884204D901240B20062100F0F2F80498FF284ED10F20062100F0EBF8D1
:204CA000012495E0287E012804D1002C02D10226344674E02046304371D102AA0499D07815
:204CC00000F088F900F0D3F8099B0BAA0A9713700698243A0C90D6789279099203AA577823
:204CE0000024002804D10621012000F0C4F801240BA90878402808D8082810D92868C0791C
:204D0000002802D00A98400009D40621032000F0B2F80124FF21304600F05CF94AE0002CA0
:204D2000F8D100970AAB0998324601900598294600F00FF93EE0002C4AD102A8C4700471F8
:204D400044718471C4710794089400F08CF803A80130019001300090811E431CC21E28464F
:204D600000F078F90646012819D003AA107800F00BF903AA0590107800F014F9054605989C
:204D8000294600F079F8022801D0012408942868C079002886D1780084D50124079400F0BE
:204DA00066F8002C00D13446012E03D10621022000F061F80898002803D00621084600F089
:204DC0005AF80798002803D00B20062100F053F820460DB0F0BD70B5074C206060C8A8685A
:204DE00031460860284600F0A2F8284600F0BDF80120207170BD07E0445E0008FFFFFFBF9D
:204E0000FF070000FFFFFF1F72B6704762B6704770B585B01E466B46044600790D461146E6
:204E20002A7E033300F0DBF804A92079039608706946C87801A948730A98019009A80078CA
:204E4000087103A8FFF7D2F805B070BD30B5054600F0B4F8FF210446284600F0BBF82046DF
:204E6000FFF7E8F830BD00B5FFF7C5FF00BD00B5FFF7CCFF00BD704710B5497A0124012982
:204E800003D30FD0032902D307D000240AE000F051F9022806D1044604E000F04BF90328AF
:204EA00000D10446204610BD70B505460E460024FFF7D9FF284600F03DF901280BD12846E7
:204EC00000F0B5F90446707A022804D101207072284600F0A5F9FFF7CAFF204670BDF0B50B
:204EE000174600240E46054600F02EFB002805D03A463146284600F039FB04462046F0BD96
:204F000000B500F03DFC00BD00B500228A720A460968012300F039F900BD00B500220A7608
:204F2000CA720A460968002300F02FF900BD10B50C460021217600F073F90120607210BD91
:204F40000E49085C70470E49085C70470D49085C704710B582B005AC2478019404AC2478D7
:204F6000009400F099FC02B010BD10B5044600F077FC204600F08EFB10BD00BF0012041096
:204F80001012041018120410694A014613682022D25C824204D9542041431868401800E067
:204FA00000207047624A13682022D25C824203D941015868401800E0002070475C4A1368B1
:204FC0002422D25C002A03D001461869405C00E010467047564B1A68126911547047FCB5A4
:204FE00081B00192524A0090012017682122D65D002E2DD0002415E001B435196D10AB003C
:20500000D3181A780198824201BC0AD806D39B788B4206D802D32C462E4603E06C1CA4B204
:2050200000E02E46BA68B442E6D3A40014192278009B9A420CD1A2788A4209D10199002909
:2050400002D1E178012903D0029A61781170002001B0FCBDF0B582B0354F01243D68242638
:20506000765D002E16D02035AE78002E08D0864210D8ED78AD19A8420CDA801BC0B202E02E
:20508000ED78A84206D2089D0195079D009500F022F80446204602B0F0BD70B5002113E023
:2050A000DB680A01D3181A7890420BD15A689B689B1805E01E4E34682469FF25A554013235
:2050C0009342F7D80131C9B2194A13682322D25C8A42E5D870BDF0B5154C2668F668000185
:2050E000855D0D702568069FED682D18A97B39702568059FED682D18697B39702568ED687E
:205100002D18297B19702168CB681B1859689B685B18022007E025682D696D5CFF2D01D104
:20512000117000200131994201D20228F3D0F0BD445E000800B55021095C406A00F0C3F8CA
:205140000146C00703D4890603D4022002E0012000E0032000BD30B50D465021095C406A67
:2051600000F0B1F80446C0070DD4FFF77CFE687A012804D10320A10600D402206872FFF7C4
:2051800076FE012000E0002030BDF9B584B0456A503005930678174600220C46B9880392BF
:2051A000002900D121882279013AD2B20192A279013AD2B200926279531EDBB24A1E92B26E
:2051C0003146284600F09BF8227BFF2A05D0012003903146284600F095F9F988002900D13A
:2051E000218A227A013AD2B20192A27A013AD2B20092627A531EDBB24A1E039892B20290F6
:205200003146284600F097F8E37A059A3146284600F0D8F804983946FFF79DFF04B0F9BD72
:2052200000B55021095C406A00F0B0F800BD00B55021095C406A00F05CF800BD0000014964
:2052400008787047485E00084902081802657047002A01D1012202E0012A04D10222490270
:20526000081898231A50704749020818F4300068C0B2704781B049020818F43000686A463A
:205280000090507801B0704749020818006D704710B549020C189C22105900F074FBC0B293
:2052A00020280CD39822105900F06DFBC0B2FF21202802D21F21091AC9B2084602E03F2130
:2052C000081AC0B210BD490208188069704749020918DC235858D83109688843D040C0072B
:2052E000C00F704749020818C4300068C002C00E704749020818406C0006C00F704730B592
:2053000081B08B4D2C6805AD00942D786C02D205D20D6D4622436A806B70009A04AD7F2317
:205320002D789A436B065B0E1A43490208180092C26101B030BD70B581B07E4E1F24240469
:205340003568A543D406E40A25436E460095737005AE3678320106AE367833071B0F6E465E
:205360001A433270009B012207AED20536789343F207120A1343490208180093C36001B023
:2053800070BD4902081880231A50704782B049020918886900906B460120187000988861B7
:2053A0000622FF3288690190C0B2012801D0013AF8D2886900906A4603201070009888614C
:2053C00002B0704770B581B05B4E3468032634432025AC43D507AD0E2C435A000126164315
:2053E000032212029443B207920D14434902081800948461816989088900816101B070BD46
:20540000000081B049020818AC2319586B4600911A800099AC23195001B0704730B581B085
:20542000464D2C6800940725AC432A401443702294435A07520E14432A0204AD2D789443FB
:205440006A07520D144349020818BC252C5001B030BD10B581B049020818842421586C468B
:2054600000912280A37000998424215001B010BD81B049020818F82319586B4600911A70C2
:205480000099F823195001B0704710B581B06C46A27023800122E270490208180099F0249D
:2054A000215001B010BD4902081801219140D02319507047F0B581B09206920E204E4025AB
:2054C00015437F223468120694432A0614436E46009406AFB3703F8837804902081800991F
:2054E000C026315001B0F0BD81B049020818C82319586B4600911A700099C823195001B085
:205500007047000010B581B00E4C4902081823686C46009362700099816401B010BD8A08E9
:20552000920089071058C90EC840C0B2704700BF14130410181304101C1304102413041012
:20554000281304102C13041030B50D4600245021095C406AFFF798FE2A7E8249012A00D1D2
:205560008149084000D00124204630BDF6B59AB01B92436A0746503004930678794A0020BD
:20558000099031461846FFF75FFE04983146FFF77FFE079040200590079C3F2C6AD8788DE3
:2055A000BD6900222D1829200692C05DFFF7CBFC0830C0B260432C582D18600002D4E00077
:2055C000440D06E0E000C0080124E40704438022069228460621FFF7A2FF830608D50123A5
:2055E0009B071C430007000FFFF7AAFC039006E00107090F0391082901D908210391284695
:205600000721FFF78CFF4006069A400E0243D2B20692039A9008C0B2930701D00130C0B297
:20562000002309E008B40BA9099199004A19099B9268CA5008BC01338342F3D31B980290D8
:205640000AA80190039823460090069A1A993846FFF7DEFB079A04983146FFF7F9FD049897
:205660003146FFF715FE059D0790013DEDB20595002D91D104983146FFF706FE8822104064
:2056800005D004983146FFF7DFFD0120099009981AB0F6BDF0B589B0344D06465036476A96
:2056A0003178029703913F2204463846FFF769FE21462831487800903B20035D3120025D13
:2056C000019103993846FFF7A9FE616A07913078618A0690A069002641180891218A4218CF
:2056E00023483746234900680592884202D10120214A01E03046214A04920699019B287003
:2057000007985A88FFF77DFE35461FE0079806992A46FFF79DFDA8000499072240580028B1
:2057200009D4B10000042843D2061043089A01368850F6B208E0F90052071043059A8850E4
:20574000501845600137FFB20135EDB201990878A842DBD80298628A03993346FFF779FEBF
:2057600009B0F0BD11000800110008186D5E0008040800080101FEFEF0100410E810041074
:20578000F0B584B00646503604463178406AFFF77BFD0290C00428D5606A009037782025B2
:2057A0001BE000983946FFF765FD0190C000C11DE089A2698018FFF7B2FE012212030390D3
:2057C00000983946FFF740FD019A00983946FFF74FFE0398FFF73AFBEDB200983946FFF718
:2057E00043FD002801D9013DDBD20299480535D54620656A035D0195029301223678920265
:2058000031462846FFF720FD002524E02A4601983146FFF75CFD00281BD02946204600F0C0
:20582000A3F807460721FFF77AFEFFF7C7FBFF280FD038460621FFF772FE0207120F039262
:2058400038460621FFF76BFE800602D50398FFF777FB0135EDB20298A842D7D804B0F0BD7B
:2058600070B581B0456A04465030E3890678227B31462846FFF709FE4434A0880090A378A5
:20588000A27931462846FFF715FEE27831462846FFF72AFE01B070BDF6B584B00BA905929A
:2058A0000F78416A06465030029101781D460191996818680391002802D44005C40804E0E1
:2058C000C000C0080124A40704434620805DB84204D801990298FFF705FD07460097394681
:2058E000304600F041F80646059A346010060124E40504432879FFF729FB049A030717683D
:205900001B0B1C43FB79012B0AD12B685B0007D501235B051C43FB7A012B01D11B051C43E8
:2059200074600836FFF70CFB002313E0002427462979FA18914202DD0399895C01E00CAA33
:205940001178FA0091400C430137042FF0D310C60433DBB28342E9D36A460BCA0246184630
:20596000FFF7A1FD04B0F6BD70B585690446463040780E46FFF7E7FA083070434834218866
:205980000818281870BD2021004202D0491E4008FCD108007047000010B5304C20780028E9
:2059A00004D1042000F060F80120207010BD10B52A4C2078002804D0042000F0A7F8002086
:2059C000207010BD254908787047F0B581B00E46224A00230093117801293BD1002839D188
:2059E0001F4C204D204600F099F8217900278F420FD27800815B207800F000F901372179CE
:205A0000FFB28F42F5D3207800F00EF900280FD10CE0207800F008F9002809D106E02078B0
:205A20002179013D00F000F9002801D1002DF6D120790027874209D2207800F0E6F8790074
:205A4000013788532079FFB28742F5D3002D01D001210091009801B0F0BD00BF6F5E00081D
:205A6000044A0008FFFF000010B584B0A24AA34B010489181A68A24B00921A68A14B019257
:205A80001A68A14B02921A6803920A68520052080A60009A03239B039A430123DB031A43CB
:205AA00003231B069A43994C81231B061A430092019A10231A4303231B069A430123DB07D4
:205AC0001A4301922268FF231B029A430F231B021A4322608E4C0123DB0722681A438D4B63
:205AE0001A43920A92020D231A43029222608A4A800083181868800A80020D221043186001
:205B0000019808620098086004B010BD7A490004411808684000400808607047F0B584B0F1
:205B20000178754A090489180A6A03231B020092CA5801235B020192CA5802920A68039243
:205B40000A68520052080A6042790924012A00D10424039A0F239A4322430123DB071A433D
:205B600003928279C3795400DB07DB0F1C436B46C4CB0C239A43A30744781B0F1A4303237B
:205B80009B069A43A3071B0905791A430024012D00D90124530832465B0023430126FF369E
:205BA000047AB243E607F60D80783243461E1F208243F006C00E02430126FF36B743E60761
:205BC000F60D37431F24A7430743029701920B6201980322120288500298012252026B1EF4
:205BE000C127BF008850C859FF2290431A06120E1043C8510398086004B0F0BD3E4A000475
:205C0000801809239B01C15070473B49000440180D22920180587047374900044018406AA5
:205C2000C007C01701307047334A000480186123DB00C058C005C00D884201D0002000E021
:205C4000012070472C4900044018016849004908C1239B000160C158012212041143C15001
:205C60002E4AC1581140C15001680122D20711430160704710B5204A000480184B1E11D348
:205C8000026852005208C124A40002600159FF2291431A06120E1143015101680122D20769
:205CA0001143016010BD1449000440183F2292018058C007C00F70470F490004184A411879
:205CC000885801221043164A885070470A490004134A41188858400840008850704706492C
:205CE000000441183F2292018858012210433F2292018850704700BF00006040AC13041048
:205D0000B0130410B4130410B813041034100040000400400000FF03780C0040FFFFFEFF69
:205D2000C80F0000704700B500F01FF900BD00B500F069F900BD00B500F029F900BD00B55E
:205D400000F049F900BD00B500F08CF900BD00B500F06AF900BD00B500F0AEF900BD00B5EA
:205D600000F0C6F900BD000070B581B0C94E00246A46951C508029462046FFF726FE0128DD
:205D80000CD00134E4B229460020FFF71EFE012802D00A2CF5D304E00A2C02D26946488855
:205DA0000612304601B070BD30B5BB4D00244620FFF7DAFFB749884207D0B8492C72087079
:205DC0008006C00F6874012002E001202872204630BD30B5B04D00244120FFF7C5FFAD496A
:205DE000884207D0AE496C7208700006C00F2874012002E001206872204630BDB0B5A64D9B
:205E000000244620FFF7B0FFA249884204D1012028722870204617E0A24F2C72F87080069C
:205E2000C00F68744120FFF79FFF9A49884204D1012068722870204606E078716C72000694
:205E4000C00F28742C700120B0BDF0B582B006460F460024019408028021314308436A4662
:205E6000951C508029462046FFF7AFFD01280CD00134E4B229460020FFF7A7FD012802D036
:205E80000A2CF5D308E00A2C06D23046FFF76CFFB84201D101210191019802B0F0BDF0B51A
:205EA0007D4E814C25462C356F1D00206871E871E07A03221043E072E07804221043E0705B
:205EC000E0790C210843E071607A1043607260791021084360716078C021884360704120C6
:205EE0000021FFF7B2FF00283CD0E9794420FFF7ACFF002836D0E17A0420FFF7A6FF0028CF
:205F000030D0E1780220FFF7A0FF00282AD0E1790F20FFF79AFF002824D0617A1D20FFF70D
:205F200094FF00281ED061790E20FFF78EFF002818D061780120FFF788FF002812D000207C
:205F400070703920397801552120E17A0155E0786076E0796077607AE0776079E076607879
:205F6000E07501E001207070F0BD00B5FFF746FF002801D0FFF793FF00BD4749032802D979
:205F80000122002001E000220120CA72704730B5414D00281CD1032903D90120E87200207C
:205FA00017E0414CE8720322E07A904311400843E072FFF707FD012808D1E17A0420FFF752
:205FC00044FF002802D02120E17A0155002000E00120287330BD10B5002812D1FFF7F2FC35
:205FE000324C012805D10420FFF7BEFE2949884203D160788007800F04E060708007800F86
:2060000000E0002010BD704710B5274C0320E17CFFF71BFF002803D02920E17C015502E05B
:206020001D490120487310BD10B51F4C0722E07C9043042210432021884380210843E07404
:20604000FFF7C0FC01280CD1E17C0320FFF7FDFE002803D02920E17C015502E00E490120C6
:20606000487310BD10B5104C0722E07C90432421084380218843E074FFF7A4FC01281AD125
:20608000E17C0320FFF7E1FE002811D02920E17C015510E0FFFF0000705E0008BB5E0008C1
:2060A000BD5E0008B85E0008845E0008A45E00081D490120487310BD10B51C4C0722E07CEA
:2060C000904306221043A0218843E074FFF77AFC01280CD1E17C0320FFF7B7FE002803D0FA
:2060E0002920E17C015502E00F490120487310BD10B50E4C0722E07C10432021884380211D
:206100000843E074FFF75EFC01280CD1E17C0320FFF79BFE002803D02920E17C015502E0A2
:2061200001490120487310BD705E0008845E000800B5011C0A2000F003F808BC18470000A2
:2061400060B400230125021C04D10B4A002A10D060BC1047914207D3891A5B194E08B2420F
:20616000F8D252006D00F5E7012D02D052086D08F0E7181C60BC70470000000060B50E1CCE
:2061800000DC4942051C00DC4042FFF7D9FF002E00DA4942F60FED0FAE4200D0404260BC59
:2061A00008BC184700000000000000000000000000000000000000000000000000000000BC
:2061C0000000000000000000000000000000000000000000000000000000000000000000BF
:2061E00000000000000000000000000000000000000000000000000000000000000000009F
:2062000000000000000000000000000000000000000000000000000000000000000000007E
:2062200000000000000000000000000000000000000000000000000000000000000000005E
:20FD00000000000004011001010000010000000000000000000000000000000000000000CB
:20FD20000000000000000000000000000000000000000000000000000000000000000000C3
:20FD40000000000000000000000000000000000000000000000000000000000000000000A3
:20FD6000000000000000000000000000000000000000000000000000000000000000000083
:20FD8000000000000000000000000000000000000000000000000000000000000000000063
:20FDA000000000000000000000000000000000000000000000000000000000000000000043
:20FDC000000000000000000000000000000000000000000000000000000000000000000023
:20FDE000000000000000000000000000000000000000000000000000000000000000000003
:20FE00000000000000000000000000000000000000000000000000000000000000000000E2
:20FE20000000000000000000000000000000000000000000000000000000000000000000C2
:20FE40000000000000000000000000000000000000000000000000000000000000000000A2
:20FE6000000000000000000000000000000000000000000000000000000000000000000082
:20FE8000000000000000000000000000000000000000000000000000000000000000000062
:20FEA000000000000000000000000000000000000000000000000000000000000000000042
:20FEC000000000000000000000000000000000000000000000000000000000000000000022
:20FEE000000000000000000000000000000000000000000000000000000000000000000002
:20FF00000000000000000000000000000000000000000000000000000000000000000000E1
:20FF20000000000000000000000000000000000000000000000000000000000000000000C1
:20FF40000000000000000000000000000000000000000000000000000000000000000000A1
:20FF6000000000000000000000000000000000000000000000000000000000000000000081
:20FF8000000000000000000000000000000000000000000000000000000000000000000061
:20FFA000000000000000000000000000000000000000000000000000000000000000000041
:20FFC000000000000000000000000000000000000000000000000000000000000000000021
:20FFE000000000000000000000000000000000000000000000000000000000000000000001
:04000005100406409D
:00000001FF
